:020000040000FA
:040000009BEF20F062
:08000800056ED8CF06F0E0CF31
:1000100007F00001E9CF0DF0EACF08F0E1CF09F0D9
:10002000E2CF0AF0D9CF0BF0DACF0CF0F3CF14F017
:10003000F4CF15F0FACF16F000C00FF001C010F0A9
:1000400002C011F003C012F004C013F09DAA2CEFFF
:1000500000F09EBA48EF01F09DA032EF00F09EB094
:1000600092EF00F0A0A238EF00F0A1B2B0EF00F0E4
:100070000FC000F010C001F011C002F012C003F078
:1000800013C004F00E8E0DC0E9FF08C0EAFF09C0DE
:10009000E1FF0AC0E2FF0BC0D9FF0CC0DAFF14C0B9
:1000A000F3FF15C0F4FF16C0FAFF055007C0E0FFCC
:1000B00006C0D8FF1000F2CF0EF0F29EF76AD00F04
:1000C000F66E000EF7220900F5500EBEF28E1200F9
:1000D000000F1F2E3D4A56616B72787C7E7E7C78C5
:1000E000726B61564A3D2E1F0FFFF0E0D1C2B5A9D9
:1000F0009E948D8783818183878D949EA9B5C2D17B
:10010000E0F0F2CF0EF0F29EF76A1C0FF66E010ED1
:10011000F7220900F5500EBEF28E1200312E312E5C
:1001200031340000E92BEC2BCF0ECF6E2B0ECE6EB0
:10013000E951180803E2E96B298CEB2BEB5101081C
:1001400003E2EA2BEB6B298AEA51010805E2ED2B69
:10015000D8B4EE2BEA6B298E9E909E9038EF00F07B
:10016000EF2BEF51020801E2F081A192A19238EF4A
:1001700000F002010E6B0001F09BF099AB98030EAA
:10018000006E002EFED7AB88000C0201B6C2E9FF5C
:10019000B7C2EAFFEFCFB9F2010EB625016E000E2D
:1001A000B72101C0E9FFEA6EEFCFBAF2B9513908C1
:1001B00004E3300EB95DB86F04D0410EB95D0A0F8B
:1001C000B86FB83BBA51390804E3300EBA5DB827AE
:1001D00004D0410EBA5D0A0FB827B8C201F0000181
:1001E000000C0201AF6BB06B01010D51020803E07E
:1001F000000E016E4AD0036A02010E510D0FE96E26
:10020000010E0320EA6EEF50030805E0000E016EB8
:1002100001013BD002010E51060805E3000E016EFC
:10022000010133D00201010EB16F030E0E5DB15D0D
:1002300001E00BE2036AB1510D0FE96E010E0320DC
:10024000EA6EEF50AF27B12BF0D7AF1F020E0E5D55
:10025000036A0D0FB46F010E0320B56FB76FB4C200
:10026000B6F2000192DF01C0B0F20201AF51B05D01
:1002700008E00001F08D000E016E010106D005D0EE
:100280000201010E016E010100D0000182EF01F0B8
:100290000201AE93ABCFADF2AD51020B01E0AE83E4
:1002A000AECFACF2AC51030807E1AE818B928C80EB
:1002B0000001EC6B12D00201AC5102080DE18B92EF
:1002C0008C90000156DF020E01010D6F0201AE910C
:1002D0000001EC6B02D00201AE9102010E513F0809
:1002E00032E30001F0B92DD0036A02010E510D0F67
:1002F000E96E010E0320EA6EACC2EFFFAEA118D08A
:1003000000016FD7015210E0F089010EEA6E4D0E28
:10031000E96E010EE26E0D0EE16E400E016EE6CF4B
:10032000EEFF012EFCD703D00201AE83000106D000
:100330000001EC510A0802E20201AE8302010E2B19
:10034000000102D00201AE830201AEA304D000017D
:1003500010DF08D00201AEA104D0010E0E5D0D6FBA
:100360000E6B00019E9A38EF00F0D1808B928C903A
:100370008B948B86F095F09729968C948B888B8A3A
:100380008C828C96000E926EE10E936E800E946EAF
:10039000F00E956E969096929694A50ECD6ECD8E9B
:1003A000CF0ECF6E2B0ECE6EB150480BB509B16E8D
:1003B000B18E9D8A9D80A082C00EF212DADED8EF47
:1003C00020F00201A76703D0A86702D007D0A82BAE
:1003D000A6C2EEFFA72FFCD7A82FFAD70001000C6A
:1003E000EA6A470EE96E0201A66BA86B040EA76FBE
:1003F0000001E7DFDAEF20F002011D6B1D51030859
:100400000EE3D8901D35036A2B0FE96E000E032012
:10041000EA6E080EEC6EED52EF6A1D2BEFD700016D
:10042000DCEF20F0EA6A330EE96E0201A66BA86BDE
:10043000100EA76F0001C5DFDEEF20F0F29CF29EE8
:10044000F2BEFDD743C2A9FFA69EA69CA680A8CF58
:1004500044F2C00EF212020144C201F00001000C8D
:1004600002012C6B2C5103081CE326512C252D6F07
:10047000436F0001E3DF01C02BF2270E02012C25A0
:100480002D6F020E2E6FD8B02E2B2EC2EAFF2DC27A
:10049000E9FF020EE26E2B0EE16EE6CFEEFF2C2B93
:1004A000E1D727C200F028C201F029C202F02AC217
:1004B00003F00001FFEF02F0F29CF29EF2BEFDD7C6
:1004C0000201276B275103081CE3265127252D6FB6
:1004D000436F0001B3DF01C028F2290E0201272576
:1004E0002D6F020E2E6FD8B02E2B2EC2EAFF2DC21A
:1004F000E9FF020EE26E280EE16EE6CFEEFF272B3B
:10050000E1D7C00EF21229C200F02AC201F02BC2BC
:1005100002F02CC203F0000128EF03F03EC243F2C8
:100520008DDF01C041F2020EEA6E3F0EE96E020E4F
:10053000E26E410EE16EE6CFEEFF010E02013E25B6
:10054000426F436F00017ADF01C041F2020EEA6E92
:10055000400EE96E020EE26E410EE16EE6CFEEFF56
:1005600002013FC201F040C202F00001000C020192
:100570001D51020A000110E0030AD8B47BD0010A21
:10058000D8B4A2D0030AD8B4C5D0070AD8B4ECD0E6
:10059000010AD8B4F3D018D102011D51020869E153
:1005A0001F6B1F51030865E31E6B1E5103085FE3B9
:1005B0001F51040DF350040DF3CF22F21E51040D10
:1005C000F3502225206F1F51100DF350226B216F25
:1005D0001E51040DF350036A2125016E225103229E
:1005E0000150A90F016E000E032201C023F203C0C7
:1005F00024F2800E2025256F266F000131D724C2FA
:10060000EAFF23C2E9FF00C0EFFF01C0ECFF02C018
:10061000ECFF03C0ECFF02011F51100DF350226BE1
:10062000216F1E51040DF350036A2125016E2251E2
:1006300003220150690F016E000E032201C023F254
:1006400003C024F2C00E2025256F266F000134D789
:1006500024C2EAFF23C2E9FF00C0EFFF01C0ECFFA4
:1006600002C0ECFF03C0ECFF02011E2B9ED71F2B24
:1006700098D7ACD002011E6B1E51030824E3D8901A
:100680001E35036A2B0F016E000E032201C021F2FA
:1006900003C022F2036A1E51210FE96E000E0320EF
:1006A000EA6EEFCF23F223C23EF2000137DF22C20F
:1006B000EAFF21C2E9FF02C0ECFFED5201C0EFFFEB
:1006C00002011E2BD9D782D002011E6B1E510308D6
:1006D00020E3036A1E51470F016E000E032201C082
:1006E00021F203C022F2036A1E51250FE96E000EAB
:1006F0000320EA6EEFCF23F223C243F200019EDE15
:1007000022C2EAFF21C2E9FF01C0EFFF02011E2B56
:10071000DDD75CD002011E6B1E51030824E3D89084
:100720001E35036A5B0F016E000E032201C021F229
:1007300003C022F2036A1E511D0FE96E000E032052
:10074000EA6EEFCF23F223C23EF20001E7DE22C2BF
:10075000EAFF21C2E9FF02C0ECFFED5201C0EFFF4A
:1007600002011E2BD9D732D002013E6B0001D6DE2A
:1007700002C01CF001C01BF0020128D00A0E0201C9
:10078000436F00015BDE01C01FF202011E6B1E51B0
:10079000030819E31F530BE1036A1E51430FE96E6F
:1007A000000E0320EA6EEF50BF0BEF6E0AD0036A13
:1007B0001E51430FE96E000E0320EA6EEF50400910
:1007C000EF6E1E2BE4D702D0020100D00001000C16
:1007D000B36AB26AEF6BF091000C8B980400100EB4
:1007E000006E002EFED78B880400100E006E002EC7
:1007F000FED729840201916B915103080CE3036A2F
:100800009151430FE96E000E0320EA6EEF5080090C
:10081000EF6E912BF1D70001000C000E83B8010E92
:100820000201926F000E83BA010E9211936F000EB7
:1008300083BC010E9311946F000E83BE010E9411C0
:100840009191E8B09181000E91A1010E016E00011D
:10085000000C006A016A0201A851D890A9B10026D3
:1008600000320132A9B3002600320132A9B50026B8
:1008700000320132A9B7002600320132A9B90026A0
:1008800000320132A9BB002600320132A9BD002688
:1008900000320132A9BF0026003201320001000CF3
:1008A000020EEA6E910EE96E0201A66BA86B100EA5
:1008B000A76F000186DD020EEA6EA10EE96E02014D
:1008C000A66BA86B040EA76F00017BDDF00E956E82
:1008D0008B98020E0201A56FA5BF43D08C84040043
:1008E0000C0E006E002EFED700D083A80BD0010E98
:1008F000006EA551016E04E0D8900036012EFCD7A1
:100900000050A11383AA0BD0010E006EA551016EF9
:1009100004E0D8900036012EFCD70050A21383AC1F
:100920000BD0010E006EA551016E04E0D890003688
:10093000012EFCD70050A31383AE0BD0010E006E26
:10094000A551016E04E0D8900036012EFCD700506E
:10095000A4138C940400100E006E002EFED7A50781
:10096000BBD7A56BA5BF03D0A55103080CE3036A51
:10097000A551A10FE96E020E0320EA6EEF50010BA4
:10098000EF6EA52BEFD7180EA56FA5078C8404007A
:100990000C0E006E002EFED700D083A817D0036A7D
:1009A000026A016A010E006EA551A66F07E0D89099
:1009B0000036013602360336A62FF9D700509113C0
:1009C00001509213025093130350941383AA17D02B
:1009D000036A026A016A010E006EA551A66F07E064
:1009E000D8900036013602360336A62FF9D70050CC
:1009F000951301509613025097130350981383AC2C
:100A000017D0036A026A016A010E006EA551A66F33
:100A100007E0D8900036013602360336A62FF9D704
:100A20000050991301509A1302509B1303509C13CA
:100A300083AE17D0036A026A016A010E006EA551E7
:100A4000A66F07E0D8900036013602360336A62F8F
:100A5000F9D700509D1301509E1302509F1303506D
:100A6000A0138C940400100E006E002EFED7A55328
:100A70008CE1A56BA5BF04D0A5510308D8A0F5D083
:100A8000A5C2A8F2040EA96F0001E3DE0150036ABB
:100A9000910FE96E020E0320EA6EEFCFA6F2ECCFC3
:100AA000A7F2ECCFA8F2ECCFA9F20201A8AF20D0B8
:100AB000A5C2A8F2040EA96F0001CBDE0150036AA3
:100AC000910FE96E020E0320EA6EEFCF00F0ECCF3B
:100AD00001F0ECCF02F0EC50FF09ED52ED52ED5277
:100AE00000C0EFFF01C0ECFF02C0ECFFEC6E0201A2
:100AF000A5C2A8F2040EA96F0001ABDE0150036A83
:100B0000330F0201A66F000E0320A76FA5C2A8F243
:100B1000040EA96F00019DDE0150036A910F0201CE
:100B2000A86F020E0320A96FA7C2EAFFA6C2E9FFC1
:100B3000E26EA8C2E1FF040E016EE6CFEEFF012EC9
:100B4000FCD7036AA551430FE96E000E0320EA6E3D
:100B5000EF50FC0BEF6EA5C2A8F2040EA96F0001C6
:100B600078DE0150036A330FE96E000E0320EA6E4F
:100B7000EFCFA6F2ECCFA7F2ECCFA8F2ECCFA9F220
:100B80000201A9AF28D0036AA551A10FE96E020E98
:100B90000320EA6EEF2C1FD0036AA551430FE96EC4
:100BA000000E0320EA6EEF500109EF6EA5C2A8F215
:100BB000040EA96F00014DDE0150036A330FE96E88
:100BC000000E0320EA6EFF0EEF6EEC6EEC6E7F0EF1
:100BD000EC6E48D00201A5C2A8F2040EA96F000174
:100BE00038DE0150036A330FE96E000E0320EA6E0F
:100BF000EFCFA6F2ECCFA7F2ECCFA8F2ECCFA9F2A0
:100C00000201A9BF30D0A95307E1A85305E1A753BA
:100C100003E1A651000827E2036AA551A10FE96E7E
:100C2000020E0320EA6EEF521EE1036AA551430F44
:100C3000E96E000E0320EA6EEF500209EF6EA5C2C6
:100C4000A8F2040EA96F000104DE0150036A330FFD
:100C5000E96E000E0320EA6EFF0EEF6EEC6EEC6E96
:100C60007F0EEC6E0201A52B05D78B880001000CCE
:100C70000201906B90BF03D090510F080FE3000169
:100C8000A7DDABDD8B98C9DD015204E1F0B102D0E4
:100C90000400F9D705DE0201902BECD70001000C0F
:100CA0000201856B8551030841E3D8908535036ABD
:100CB0002B0FE96E000E0320EA6EECCF03F0ED522D
:100CC000EFCF90F203C091F2D8908535036A5B0FA5
:100CD000E96E000E0320EA6EECCF03F0ED52EF5008
:100CE00090258E6F035091218F6F8FBF0BD08F5146
:100CF0000F0808E2FF0A03E18E51000803E2100E1C
:100D00008F6F8E6B8FBF01D002D08F6B8E6BD890A0
:100D10008535036A860FE96E020E0320EA6E8FC2E4
:100D2000ECFFED528EC2EFFF852BBCD7000E956E07
:100D30008B9A8C988C9A8C9C8C9E856B8551030821
:100D40000FE38C840400100E006E002EFED78C94EE
:100D500004000C0E006E002EFED700D0852BEED7BF
:100D60000C0E856F850787C203F086C202F085519D
:100D7000006E05E0D89003320232002EFBD70250FD
:100D800002B002D08C9801D08C8889C203F088C24E
:100D900002F08551006E05E0D89003320232002E39
:100DA000FBD7025002B002D08C9A01D08C8A8BC241
:100DB00003F08AC202F08551006E05E0D89003323C
:100DC0000232002EFBD7025002B002D08C9C01D020
:100DD0008C8C8DC203F08CC202F08551006E05E050
:100DE000D89003320232002EFBD7025002B002D05C
:100DF0008C9E01D08C8E8C840400100E006E002E10
:100E0000FED78C9404000C0E006E002EFED700D08E
:100E10008553A8E18B8AF00E956E845303E00001A0
:100E200027DF02010001000C020EEA6E980EE96E47
:100E3000EF5011E0060E016EBF0E006E0400002E92
:100E4000FDD7012EF9D77A0E006E002EFED700D006
:100E50000400EF2EEFD7000C8B948B96000E956E4E
:100E60008C92040E0201846F8407036A8451470F39
:100E7000E96E000E0320EA6EEF50020B020802E159
:100E80008C8801D08C988C840400100E006E002E8B
:100E9000FED78C9404000C0E006E002EFED700D0FE
:100EA0008453E2E1040E846F8407036A8451470F80
:100EB000E96E000E0320EA6EEF50010B02E18C8810
:100EC00001D08C988C840400100E006E002EFED78A
:100ED0008C9404000C0E006E002EFED700D08453BC
:100EE000E3E18C82F00E956E190E986F00019CDF85
:100EF000BFDE8B948B86000C10C2EAFF0FC2E9FFA5
:100F0000020142C2EFFFE92AD8B4EA2AEF6A0F2BA6
:100F1000D8B4102B0001000C020141BF11D00F0EFC
:100F2000006E403900160A0E005C03E2300E002607
:100F300002D04151002600C042F20001DDDF020173
:100F40000F0E40170A0E405D02E2300E02D0419FA4
:100F50004151402740C242F20001CEDF000C010E99
:100F6000EA6E8D0EE96E0201A66BA86B800EA76F6C
:100F70000001E1EC01F0010E0201106F8D0E0F6F08
:100F80003EC240F2370E416F0001C6DF3FC240F261
:100F9000370E0201416F0001BFDF000C3FC241F27A
:100FA0003EC240F241C203F0020140C2E9FF41C229
:100FB000EAFFEF5206E0402BD8B4412B0001F2D7F4
:100FC00002013E51405D006E3F514159036E00C029
:100FD00001F0026E0001000C3C0E02012F6F435025
:100FE000400B02E0320E2F6F2D51000117E0010A75
:100FF0001BE0040A20E0030AD8B484D0010AD8B464
:10100000B2D00F0AD8B4E0D0030AD8B419D11B0A61
:10101000D8B49AD1040AD8B450D22FD302013E6B6F
:101020003F6B00019CDF2AD3010E02013E6F3F6B34
:10103000000195DF23D3050E02013E6F200E3F6FA6
:1010400000018DDF02012E6B2E51030859E3010EC2
:101050003F6F8D0E3E6F0001A1DF8D0E0201012456
:10106000306F010E0220316F2E51040DF350036AD0
:10107000330FE96E000E0320EA6EEFCF3EF2ECCFA5
:101080003FF2ECCF40F2ECCF41F23FC239F23EC228
:1010900038F22E51040DF350036A330FE96E000E3F
:1010A0000320EA6EEFCF3EF2ECCF3FF2ECCF40F2FE
:1010B000ECCF41F241C237F240C236F231C210F2F7
:1010C00030C20FF237C240F2370E416F000124DF09
:1010D00036C240F2370E0201416F00011DDF39C2F6
:1010E00040F2370E0201416F000116DF38C240F2B4
:1010F000370E0201416F00010FDF02012E2BA4D732
:101100000001BCD2060E02013E6F080E3F6F0001C7
:1011100026DF02012E6B2E51030823E3010E3F6FE1
:101120008D0E3E6F00013ADF8D0E02010124306FFB
:10113000010E0220316F036A2E51470FE96E000E37
:101140000320EA6EEFCF3EF231C210F230C20FF24E
:101150003EC240F2370E416F0001DEDE02012E2B4F
:10116000DAD700018BD2070E02013E6F080E3F6FE7
:101170000001F5DE02012E6B2E51030823E3010E60
:101180003F6F8D0E3E6F000109DF8D0E02010124BD
:10119000306F010E0220316F036A2E51430FE96E4A
:1011A000000E0320EA6EEFCF3EF231C210F230C2E1
:1011B0000FF23EC240F2370E416F0001ADDE020178
:1011C0002E2BDAD700015AD2080E02013E6F100E04
:1011D0003F6F0001C4DE02012E6B2E5103082EE387
:1011E000010E3F6F8D0E3E6F0001D8DE8D0E0201A5
:1011F0000124306F010E0220316FD8902E35036A22
:101200002B0FE96E000E0320EA6EECCF3FF2ED5299
:10121000EFCF3EF231C210F230C20FF23FC240F2C5
:10122000370E416F000178DE3EC240F2370E0201F8
:10123000416F000171DE02012E2BCFD700011ED2BB
:101240000B0E02013E6F120E3F6F000188DE6F0E23
:101250000201356F120E346F030E336F810E326F41
:101260003337323333332E6B2E51030823E3010E11
:101270003F6F8D0E3E6F000191DE8D0E0201012445
:10128000306F010E0220316F036A2E51320FE96E6A
:10129000020E0320EA6EEFCF3EF231C210F230C2EE
:1012A0000FF23EC240F2370E416F000135DE0201FF
:1012B0002E2BDAD76F0E356F120E346F030E336F8D
:1012C000800E326F3337323333332E6B2E51030897
:1012D00023E3010E3F6F8D0E3E6F00015FDE8D0E2A
:1012E00002010124306F010E0220316F036A2E517A
:1012F000320FE96E020E0320EA6EEFCF3EF231C2EA
:1013000010F230C20FF23EC240F2370E416F0001C0
:1013100003DE02012E2BDAD7010E3F6F8D0E3E6FDA
:1013200000013CDE8D0E02010124306F010E02200F
:10133000316F31C210F230C20FF20C0E406F370E17
:10134000416F0001E9DD9AD1100E02013E6F180EC7
:101350003F6F000104DE010E02013F6F8D0E3E6FF4
:1013600000011CDE8D0E02010124306F010E0220EF
:10137000316F31C210F230C20FF20C0E406F370ED7
:10138000416F0001C9DD200E0201406F370E416F31
:101390000001C2DD010E02013F6F8D0E3E6F0001A4
:1013A000FDDD8D0E02010124306F010E0220316F30
:1013B00031C210F230C20FF2050E406F370E416F8E
:1013C0000001AADD010E02013F6F8D0E3E6F00018C
:1013D000E5DD8D0E02010124306F010E0220316F18
:1013E00031C210F230C20FF23E6B3E51000181EC6F
:1013F00000F0000908E002013E2B426F00017CDD95
:101400000201F3D70001010E02013F6F8D0E3E6F06
:101410000001C4DD8D0E02010124306F010E022097
:10142000316F3E6B00018EEC02F002C037F201C05A
:1014300036F231C210F230C20FF237C240F2370E2C
:101440000201416F000168DD36C240F2370E020131
:10145000416F000161DD0201356B346B336B7D0E32
:10146000326F3337323333332E6B2E51030823E37D
:10147000010E3F6F8D0E3E6F000190DD8D0E02015B
:101480000124306F010E0220316F036A2E51320F9A
:10149000E96E020E0320EA6EEFCF3EF231C210F287
:1014A00030C20FF23EC240F2370E416F000134DD10
:1014B00002012E2BDAD70001E1D0140E02013E6F9B
:1014C0001E0E3F6F00014BDD010E02013F6F8D0EBE
:1014D0003E6F000163DD8D0E02010124306F010EAD
:1014E0000220316F31C210F230C20FF2040E406F91
:1014F000370E416F000110DD010E02013F6F8D0EAE
:101500003E6F00014BDD8D0E02010124306F010E94
:101510000220316F31C210F230C20FF2180E406F4C
:10152000370E416F0001F8DC0201356B400E346F5D
:101530001C0E336F800E326F3337323333332E6BE2
:101540002E51030823E3010E3F6F8D0E3E6F000105
:1015500025DD8D0E02010124306F010E0220316F56
:10156000036A2E51320FE96E020E0320EA6EEFCFAE
:101570003EF231C210F230C20FF23EC240F2370EDC
:10158000416F0001C9DC02012E2BDAD7356B346BB9
:10159000480E336F780E326F3337323333332E6B5E
:1015A0002E51030823E3010E3F6F8D0E3E6F0001A5
:1015B000F5DC8D0E02010124306F010E0220316F27
:1015C000036A2E51320FE96E020E0320EA6EEFCF4E
:1015D0003EF231C210F230C20FF23EC240F2370E7C
:1015E000416F000199DC02012E2BDAD7356B346B89
:1015F000336B7D0E326F3337323333332E6B2E51D4
:10160000030823E3010E3F6F8D0E3E6F0001C6DC21
:101610008D0E02010124306F010E0220316F036A2A
:101620002E51320FE96E020E0320EA6EEFCF3EF22A
:1016300031C210F230C20FF23EC240F2370E416F9B
:1016400000016ADC02012E2BDAD7010E3F6F8D0EEE
:101650003E6F0001A3DC8D0E02010124306F010EEC
:101660000220316F31C210F230C20FF22FC240F2AD
:10167000370E416F000150DC01D000D0000C020198
:10168000306B2F6B010E3F6F8D0E3E6F000186DCBD
:1016900002C003F00150035205E1015002012F5D29
:1016A0000DE20001036A02012F518D0FE96E010E58
:1016B0000320EA6EEF5030272F2BE4D7301F30C2C3
:1016C00001F0000199EF0BF00400020131519EA8D6
:1016D000FED7AD6EACB202D00400FCD70001000C06
:1016E000020130BF11D00F0E006E2F3900160A0E06
:1016F000005C03E2300E002602D03051002600C00C
:1017000031F20001E1DF02010F0E2F170A0E2F5DEB
:1017100002E2300E02D0309F30512F272FC231F21B
:101720000001D2DFC2EF0BF002012D6B2E6B000126
:10173000A6D701C02EF2020E0201316F0001C4DFF4
:10174000036A02012D518D0FE96E010E0320EA6E2E
:10175000EF5212E0036A2D518D0FE96E010E032046
:10176000EA6EEFCF2FF22FC231F20001ADDF02019E
:101770002D2B0001E5D702012EC22FF2370E306F5C
:101780000001AED7030E0201316F00019DDF000C96
:101790000201836B8351030838E3D8908335036AD1
:1017A0002B0F016E000E032203C085F2D890833503
:1017B000036A7F25E96E80510320EA6EECCF03F0C7
:1017C000ED52EFCF86F285C2EAFF01C0E9FF03C008
:1017D000ECFFED5286C2EFFF036A8351470F016EA3
:1017E000000E032203C085F2036A83518125E96E4E
:1017F00082510320EA6EEFCF86F285C2EAFF01C074
:10180000E9FF86C2EFFF832BC5D7010E846F00016D
:1018100050EC06F02CEC07F0000C02018A518E19F6
:10182000800B946F8AAF0BD0871F881F891F8A1F78
:10183000872BD8B4882BD8B4892BD8B48A2B8EAFF9
:101840000BD08B1F8C1F8D1F8E1F8B2BD8B48C2B16
:10185000D8B48D2BD8B48E2B006A016A026A036A51
:101860008F6B906B916B926B8E518D118C118B11D4
:101870002CE0200E936FD8908737883789378A37C6
:101880008F379037913792378E51925D08E18D51A5
:10189000915D05E18C51905D02E18B518F5D0FE30D
:1018A0008B518F5F8C51D8A08C3D905F8D51D8A00B
:1018B0008D3D915F8E51D8A08E3D925FD8800036CD
:1018C000013602360336932FD6D794AF0BD0001EC5
:1018D000011E021E031E002AD8B4012AD8B4022A0F
:1018E000D8B4032A020EEA6E8F0EE96E0001000CD6
:1018F0008E0E006E80C201F07FC202F0036A01AE5C
:1019000005D0011E021E022A01E1012A015209E14D
:1019100002C001F0026A080E005E015202E1006A94
:101920000DD0D89001BE04D0023601360006F9D79A
:10193000020180AF02D0000101D0019E0001000C25
:1019400002018351D8B4A5D08F6F8751D8B4A1D0EC
:101950008F5F05E37F0E8F27D8B09BD006D0810E16
:101960008F5FD8A096D0D8B494D08FC200F0016A0F
:10197000026A036A8E6B84C28DF28D8F85C28CF2EF
:1019800086C28BF2190E8F6F8A518B5F0DE2010EAA
:101990008C5F0AE28D5F08E28E5F06E28E2B8D2B54
:1019A0008C2B8A518B2728D089518C5F12E2010E33
:1019B0008D5F0FE28E5F0DE28E2B8D2B89518C2770
:1019C0008A518B2719E38C2B17E18D2B15E18E2B78
:1019D00013D0885180098D5F0EE2010E8E5F0BE2FD
:1019E0008E2B885180098D2789518C27E9E38D2B17
:1019F000E7E18E2BE5D703808F2F01D00BD0D89055
:101A00008B378C378D378E37D890033602360136B8
:101A10009037BAD790A106D0D89001320232033263
:101A2000903302D0000635E090BF1ED0D8908B379F
:101A30008C378D378E378A518B5F07E2010E8C5FB2
:101A400004E28D5F02E28E5F1AE389518C5F05E24A
:101A5000010E8D5F02E28E5F12E3885180098D5F77
:101A600003E2010E8E5F0BE3032A09E1022A07E17C
:101A7000012A05E1002A0DE001320232033284C25C
:101A80008FF288518F1B8FAF02D0018E06D0019E3E
:101A900004D0006A016A026A036A0001000CF29C29
:101AA000F29EF2BEFDD796C2A9FF97C2A8FFA69CE0
:101AB000A69EA684F2CF00F0F29E0F01550EA76EEF
:101AC000AA0EA76EA682A6B2FED7A6940050F21266
:101AD000050E0201986F000114EC07F0C00EF2121F
:101AE000000C02018F6B8FBF03D08F5103081CE3E2
:101AF000036A8F518B0F956F020E0320966F020EB3
:101B0000EA6E900EE96E96C2E2FF95C2E1FFE6CF63
:101B1000EEFF8A518F25956F966F90C297F2000164
:101B2000BEDF02018F2BDFD7000125EF0EF002018F
:101B30008F6B8F5103081CE38B0E8F25916F020E64
:101B4000926FD8B0922B020EEA6E900EE96E92C29E
:101B5000E2FF91C2E1FFE6CFEEFF8A518F25916F40
:101B6000966F90C297F200019ADF02018F2BE1D7A6
:101B7000000150EF0EF0020EEA6E890EE96E020EC1
:101B8000E26E870EE16EE6CFEEFF86C296F289C264
:101B900097F285DF020EEA6E890EE96E020EE26EA2
:101BA000880EE16EE6CFEEFF010E020186258C6FF6
:101BB000966F89C297F2000172DF000C02017F511B
:101BC000FA0FD8B000D1060F0001E5EF0EF00201C8
:101BD000816B8151030869E3806B8051030863E3E3
:101BE0008151040DF350040DF3CF84F28051040DA4
:101BF000F3508425826F800E8225836F8151100DF2
:101C0000F350856B846F8051040DF350036A842573
:101C1000016E855103220150A90FE96E000E0320C9
:101C2000EA6EEFCF86F2ECCF87F2ECCF88F2ECCF02
:101C300089F283C28AF289C28EF288C28DF287C28B
:101C40008CF286C28BF200014CD7C00E02018225B5
:101C5000836F8151100DF350856B846F8051040D9B
:101C6000F350036A8425016E855103220150690FE8
:101C7000E96E000E0320EA6EEFCF86F2ECCF87F21A
:101C8000ECCF88F2ECCF89F283C28AF289C28EF25D
:101C900088C28DF287C28CF286C28BF2000147D7D0
:101CA0000201802B9AD7812B94D78DD00201806BB3
:101CB0008051030821E3036A8051210FE96E000E71
:101CC0000320EA6EEFCF83F2D8908035036A2B0FA2
:101CD000E96E000E0320EA6EECCF85F2ED52EFCFF5
:101CE00084F283C286F285C288F284C287F2000140
:101CF00042DF0201802BDCD766D00201806B80516D
:101D000003081BE3036A8051250FE96E000E0320D0
:101D1000EA6EEFCF83F2036A8051470FE96E000E3F
:101D20000320EA6EEFCF84F283C296F284C297F268
:101D30000001B5DE0201802BE2D745D00201806BA5
:101D40008051030821E3036A80511D0FE96E000EE4
:101D50000320EA6EEFCF83F2D8908035036A5B0FE1
:101D6000E96E000E0320EA6EECCF85F2ED52EFCF64
:101D700084F283C286F285C288F284C287F20001AF
:101D8000FADE0201802BDCD71ED00201866B1CC05C
:101D900088F21BC087F20001EEDE020114D043502E
:101DA000400B07E10A0E0201966F976B000177DE88
:101DB00007D00A0E0201966F010E976F00016FDEC9
:101DC000020101D002010001000CF2CF0EF0F29EE0
:101DD000E824F76AF736EF0FF66E1D0EF7220A00B9
:101DE000F550FA6E0800F5500EBEF28EF96EFA1C30
:101DF000AC1CCE1B3C1D8A1D9E1D02012D6B2D515E
:101E0000030838E3D8902D35036A730F016E020E74
:101E1000032203C080F2D8902D35036A2B0FE96EA0
:101E2000000E0320EA6EECCF03F0ED52EFCF81F20B
:101E300080C2EAFF01C0E9FF03C0ECFFED5281C29E
:101E4000EFFF036A2D517B0F016E020E032203C0C8
:101E500080F2036A2D51470FE96E000E0320EA6EEF
:101E6000EFCF81F280C2EAFF01C0E9FF81C2EFFF3C
:101E70002D2BC5D72D6B2D5103080CE3036A2D5173
:101E8000430FE96E000E0320EA6EEF50FB0BEF6E7E
:101E90002D2BF1D72D6B2D51030837E32F6B2F51CD
:101EA000030831E32F51100DF350806B7F6F2D51DC
:101EB000040DF350036A7F25016E80510322015007
:101EC000690FE96E000E0320EA6E7F0EEF6EEC6A7A
:101ED000EC6AEC6A2F51100DF350806B7F6F2D511F
:101EE000040DF350036A7F25016E805103220150D7
:101EF000A90FE96E000E0320EA6EEF6AEC6AEC6A45
:101F0000EC6A2F2BCCD72D2BC6D78B928C902F6BB6
:101F10002F510308D8A041EF15F08B948B962D6BB1
:101F20002D51030829E32D51040DF350036A310F9D
:101F3000E96E020E0320EA6EEF6AEC6AEC6AEC6A64
:101F40002D51040DF350036A410FE96E020E032078
:101F5000EA6EEF6AEC6AEC6AEC6A2D51040DF350FC
:101F6000036A510FE96E020E0320EA6EEF6AEC6A13
:101F7000EC6AEC6A2D2BD4D72F51FC0FD8B084D04B
:101F8000040F000156EF15F002012D6B2D510308CF
:101F90000AE3036A2D51470FE96E000E0320EA6E33
:101FA000EF6A2D2BF3D7FF0E646FFE0E636FB70E33
:101FB000626FE00E616F686B010E676F480E666FAF
:101FC000200E656F61D002012D6B2D5103080BE3CC
:101FD000036A2D51470FE96E000E0320EA6E020ED0
:101FE000EF6E2D2BF2D7FF0E646FFA0E636FDF0ECC
:101FF000626F800E616F686B050E676F200E666FF3
:10200000800E656F41D002012D6B2D5103080BE34B
:10201000036A2D51470FE96E000E0320EA6E010E90
:10202000EF6E2D2BF2D7FF0E646FFE0E636FB70EAF
:10203000626FE00E616F686B010E676F480E666F2E
:10204000200E656F21D002012D6B2D5103080BE38B
:10205000036A2D51470FE96E000E0320EA6E030E4E
:10206000EF6E2D2BF2D7FF0E646FFA0E636FDF0E4B
:10207000626F800E616F686B050E676F200E666F72
:10208000800E656F01D002012D6B2D5103080EE308
:10209000D8902D35036A2B0FE96E000E0320EA6EEF
:1020A000040EEC6EED52EF6A2D2BEFD700012CECF5
:1020B00007F0010E0201846F000150EC06F00201EE
:1020C0002D6B2D510708D8A0A3D00001E8EC03F038
:1020D000EDEC03F08B980DEC04F0015204E1F0B14B
:1020E00002D00400F8D7F0A11ED002012E6B2E51B1
:1020F00004080CE3036A2E51430FE96E000E03201F
:10210000EA6EEF500409EF6E2E2BF1D7020E806FAE
:10211000730E7F6F020E826F7B0E816F0001C8EC21
:102120000BF054EF15F050EC04F002012E6B2E5121
:10213000030824E3036A2E51430FE96E000E0320C7
:10214000EA6EEF50030B18E0036A2E51430FE96E5D
:10215000000E0320EA6EEF500409EF6E020E806F4E
:10216000730E7F6F020E826F7B0E816F0001C8ECD1
:102170000BF054EF15F002012E2BD9D72E6B2E51F8
:10218000030844E32E51040DF350036A410F016E1E
:10219000020E032201C07FF203C080F22E51040D13
:1021A000F350036A410FE96E020E0320EA6EEFCF8F
:1021B00081F2ECCF82F2ECCF83F2ECCF84F22E519D
:1021C000040DF350036A330FE96E000E0320EA6E2C
:1021D000EFCF00F0ECCF01F0ECCF02F0ECCF03F04A
:1021E000815100268251012283510222845103220F
:1021F00080C2EAFF7FC2E9FF00C0EFFF01C0ECFF31
:1022000002C0ECFF03C0ECFF2E2BB9D72D2B59D702
:102210002D6B2D510308D8A0AAD02D51040DF350D9
:10222000036A410F016E020E032201C07FF203C058
:1022300080F22D51040DF350036A410FE96E020E36
:102240000320EA6EEFCF81F2ECCF82F2ECCF83F283
:10225000ECCF84F2EACF86F2E9CF85F284C28AF22B
:1022600083C289F282C288F281C287F28E6B8D6B43
:102270008C6B080E8B6F00010DEC0CF086C2EAFF30
:1022800085C2E9FF80C2EAFF7FC2E9FF00C0EFFF1D
:1022900001C0ECFF02C0ECFF03C0ECFF02012D51B6
:1022A000040DF350036A410FE96E020E0320EA6E3B
:1022B000EFCF7FF2ECCF80F2ECCF81F2ECCF82F265
:1022C00082AF03D064AF39D002D064BF0FD0825147
:1022D000645D0CE332E18151635D08E32EE18051DE
:1022E000625D04E32AE161517F5D27E32D51040D16
:1022F000F350036A410FE96E020E0320EA6EEFCF3E
:1023000083F2ECCF84F2ECCF85F2ECCF86F268AFAB
:1023100003D086AF12D002D086BF27D06851865D29
:1023200024E30BE16751855D20E307E16651845D9D
:102330001CE303E18351655D18E2036A2D51430FED
:10234000E96E000E0320EA6EEF500409EF6E020EF4
:10235000806F730E7F6F020E826F7B0E816F0001A4
:10236000C8EC0BF054EF15F002012D2B52D78B94D3
:102370008B862D6B2D5103080EE3D8902D35036A03
:102380002B0FE96E000E0320EA6E0C0EEC6EED5280
:10239000EF6A2D2BEFD7010E846F000150EC06F091
:1023A00002012D6B2D510708D8A0A1D00001E8EC47
:1023B00003F0EDEC03F08B980DEC04F0015204E116
:1023C000F0B102D00400F8D7F0A11DD002012E6BAD
:1023D0002E5104080CE3036A2E51430FE96E000EE0
:1023E0000320EA6EEF500409EF6E2E2BF1D7020E98
:1023F000806F730E7F6F020E826F7B0E816F000104
:10240000C8EC0BF051D350EC04F002012E6B2E51AE
:10241000030823E3036A2E51430FE96E000E0320E5
:10242000EA6EEF50030B17E0036A2E51430FE96E7B
:10243000000E0320EA6EEF500409EF6E020E806F6B
:10244000730E7F6F020E826F7B0E816F0001C8ECEE
:102450000BF02AD302012E2BDAD72E6B2E51030854
:1024600044E32E51040DF350036A310F016E020E46
:10247000032201C07FF203C080F22E51040DF350FD
:10248000036A310FE96E020E0320EA6EEFCF81F28C
:10249000ECCF82F2ECCF83F2ECCF84F22E51040D1C
:1024A000F350036A330FE96E000E0320EA6EEFCF9C
:1024B00000F0ECCF01F0ECCF02F0ECCF03F0815153
:1024C000002682510122835102228451032280C2BC
:1024D000EAFF7FC2E9FF00C0EFFF01C0ECFF02C0CE
:1024E000ECFF03C0ECFF2E2BB9D72D2B5BD72D6B48
:1024F0002D510308D8A0A9D02D51040DF350036A23
:10250000310F016E020E032201C07FF203C080F280
:102510002D51040DF350036A310FE96E020E0320B2
:10252000EA6EEFCF81F2ECCF82F2ECCF83F2ECCF08
:1025300084F2EACF86F2E9CF85F284C28AF283C2BE
:1025400089F282C288F281C287F28E6B8D6B8C6BAE
:10255000080E8B6F00010DEC0CF086C2EAFF85C2FD
:10256000E9FF80C2EAFF7FC2E9FF00C0EFFF01C0C0
:10257000ECFF02C0ECFF03C0ECFF02012D51040D83
:10258000F350036A310FE96E020E0320EA6EEFCFBB
:102590007FF2ECCF80F2ECCF81F2ECCF82F282AF0F
:1025A00003D064AF39D002D064BF0FD08251645DD4
:1025B0000CE332E18151635D08E32EE18051625DFD
:1025C00004E32AE161517F5D27E32D51040DF350AF
:1025D000036A310FE96E020E0320EA6EEFCF83F239
:1025E000ECCF84F2ECCF85F2ECCF86F268AF03D06B
:1025F00086AF12D002D086BF26D06851865D23E315
:102600000BE16751855D1FE307E16651845D1BE3C4
:1026100003E18351655D17E2036A2D51430FE96EB3
:10262000000E0320EA6EEF500409EF6E020E806F79
:10263000730E7F6F020E826F7B0E816F0001C8ECFC
:102640000BF032D202012D2B53D72D6B2D510308E5
:102650000EE3D8902D35036A2B0FE96E000E032090
:10266000EA6E080EEC6EED52EF6A2D2BEFD7010EDD
:10267000846F000150EC06F002012D6B2D5107080C
:10268000D8A0A1D00001E8EC03F0EDEC03F08B98AA
:102690000DEC04F0015204E1F0B102D00400F8D7CF
:1026A000F0A11DD002012E6B2E5104080CE3036A29
:1026B0002E51430FE96E000E0320EA6EEF5004091D
:1026C000EF6E2E2BF1D7020E806F730E7F6F020E0E
:1026D000826F7B0E816F0001C8EC0BF0E5D150ECEE
:1026E00004F002012E6B2E51030823E3036A2E51DE
:1026F000430FE96E000E0320EA6EEF50030B17E064
:10270000036A2E51430FE96E000E0320EA6EEF506C
:102710000409EF6E020E806F730E7F6F020E826FE0
:102720007B0E816F0001C8EC0BF0BED102012E2B95
:10273000DAD72E6B2E51030844E32E51040DF350CB
:10274000036A510F016E020E032201C07FF203C023
:1027500080F22E51040DF350036A510FE96E020E00
:102760000320EA6EEFCF81F2ECCF82F2ECCF83F25E
:10277000ECCF84F22E51040DF350036A330FE96E4F
:10278000000E0320EA6EEFCF00F0ECCF01F0ECCFAB
:1027900002F0ECCF03F081510026825101228351D7
:1027A00002228451032280C2EAFF7FC2E9FF00C0F7
:1027B000EFFF01C0ECFF02C0ECFF03C0ECFF2E2BCB
:1027C000B9D72D2B5BD72D6B2D510308D8A0A9D0DD
:1027D0002D51040DF350036A510F016E020E0322B6
:1027E00001C07FF203C080F22D51040DF350036A43
:1027F000510FE96E020E0320EA6EEFCF81F2ECCFAB
:1028000082F2ECCF83F2ECCF84F2EACF86F2E9CF0A
:1028100085F284C28AF283C289F282C288F281C2BE
:1028200087F28E6B8D6B8C6B080E8B6F00010DEC3D
:102830000CF086C2EAFF85C2E9FF80C2EAFF7FC2D0
:10284000E9FF00C0EFFF01C0ECFF02C0ECFF03C0D6
:10285000ECFF02012D51040DF350036A510FE96E94
:10286000020E0320EA6EEFCF7FF2ECCF80F2ECCFC6
:1028700081F2ECCF82F282AF03D064AF39D002D0C4
:1028800064BF0FD08251645D0CE332E18151635D1E
:1028900008E32EE18051625D04E32AE161517F5D2E
:1028A00027E32D51040DF350036A510FE96E020E18
:1028B0000320EA6EEFCF83F2ECCF84F2ECCF85F207
:1028C000ECCF86F268AF03D086AF12D002D086BFBD
:1028D00026D06851865D23E30BE16751855D1FE3D8
:1028E00007E16651845D1BE303E18351655D17E2F7
:1028F000036A2D51430FE96E000E0320EA6EEF507C
:102900000409EF6E020E806F730E7F6F020E826FEE
:102910007B0E816F0001C8EC0BF0C6D002012D2B9D
:1029200053D72D6B2D510308D8A0A8D02F51100DCF
:10293000F350806B7F6F2D51040DF350036A7F2598
:10294000016E805103220150A90F016E000E032277
:1029500001C081F203C082F22D51040DF350036ACD
:10296000510FE96E020E0320EA6EEFCF00F0ECCFBC
:1029700001F0ECCF02F0ECCF03F082C2EAFF81C29B
:10298000E9FF00C0EFFF01C0ECFF02C0ECFF03C095
:10299000ECFF2D51040DF350036A310FE96E020E66
:1029A0000320EA6EEFCF00F0ECCF01F0ECCF02F0A5
:1029B000ECCF03F001C06CF200C06BF22D51040D9E
:1029C000F350036A410FE96E020E0320EA6EEFCF67
:1029D00000F0ECCF01F0ECCF02F0ECCF03F001C03F
:1029E0006EF200C06DF26D516B5D006E6E516C59F0
:1029F000036E00C07FF2806F000178EC0CF000C025
:102A00007FF201C080F202C081F203C082F203C0F3
:102A100086F202C085F201C084F200C083F2020196
:102A20008A6B896B886B8A0E876F0001A0EC0CF0B3
:102A300003C072F202C071F201C070F200C06FF206
:102A400002012F51100DF350806B7F6F2D51040D3B
:102A5000F350036A7F25016E805103220150690FF4
:102A6000E96E000E0320EA6E6FC2EFFF70C2ECFF4A
:102A700071C2ECFF72C2ECFF2D2B54D72F2B88EFC5
:102A80000FF0020E806F730E7F6F020E826F7B0E4F
:102A9000816F0001C8EC0BF0020E02017F6F000194
:102AA000DEEC0DF08B928C8036EF19F0F2CF0EF049
:102AB000F29EE824F76AF736D10FF66E2A0EF72257
:102AC0000A00F550FA6E0800F5500EBEF28EF96E4F
:102AD000881F0620C61F4620D89002012D35036AA4
:102AE0005B0FE96E000E0320EA6EEC6AED52EF6AAE
:102AF000D8902D35036A2B0FE96E000E0320EA6E85
:102B0000ECCF03F0ED52EFCF3EF203C03FF2036A89
:102B10002D51470FE96E000E0320EA6EEFCF48F209
:102B2000036A2D51470FE96E000E0320EA6EEF6A2B
:102B300000012CEC07F0036A02012D51430FE96EEE
:102B4000000E0320EA6EEF50F70BEF6E49914993A8
:102B500049857F0E316FFF0E306F2F6F2E6F8B9276
:102B60008C90070E416FE20E406F41510808D8A0CB
:102B70000FD104E140511E08D8A00AD18B948B9646
:102B8000D8902D35036A2B0FE96E000E0320EA6EF4
:102B900041C2ECFFED5240C2EFFF4051E2080AE1B2
:102BA0004151070807E1010E846F000150EC06F067
:102BB00005D00201846B000150EC06F0190E0201F1
:102BC000986F000114EC07F08B948B86E8EC03F00F
:102BD000EDEC03F08B980DEC04F0015204E1F0B140
:102BE00002D00400F8D7F0A10DD0036A02012D51E4
:102BF000430FE96E000E0320EA6EEF500809EF6EF6
:102C0000C7D0000150EC04F0036A02012D51430FBC
:102C1000E96E000E0320EA6EEF50030B07E07F0E13
:102C2000356FFF0E346F336F326F1AD049812D51DB
:102C3000040DF350036A330FE96E000E0320EA6EB1
:102C4000EFCF00F0ECCF01F0ECCF02F0ECCF03F0CF
:102C500003C035F202C034F201C033F200C032F2D8
:102C60004051E2080BE14151070808E135C239F251
:102C700034C238F233C237F232C236F23251365DE4
:102C80004A6F335137594B6F345138594C6F355166
:102C900039594D6F4AC200F04BC201F04CC202F0EC
:102CA000036EE8AE0DD0000ED8804A55006E000EBF
:102CB0004B55016E000E4C55026E000E4D55036EC5
:102CC00003C04EF202C04DF201C04CF200C04BF204
:102CD00003BE18D04E530AE14D5308E14C514F0842
:102CE00011E2FF0A03E14B5100080CE2363D07D028
:102CF000373D05D0383D03D039517F0803E049B353
:102D000001D0498332C200F033C201F034C202F074
:102D100035C203F035AF0DD0000ED8803255006EAD
:102D2000000E3355016E000E3455026E000E3555FF
:102D3000036E03C03DF202C03CF201C03BF200C092
:102D40003AF235C239F234C238F233C237F232C203
:102D500036F23D51315D18E30BE13C51305D14E337
:102D600007E13B512F5D10E303E12E513A5D0CE288
:102D70003DC231F23CC230F23BC22FF23AC22EF2D7
:102D800041C247F240C246F2402BD8B4412BEDD6A7
:102D900049A102D049B30AD0036A2D51430FE96E0D
:102DA000000E0320EA6EEF500809EF6E4651E2086C
:102DB00003E14751070806E046511E080DE147515F
:102DC00008080AE1036A2D51430FE96E000E032043
:102DD000EA6EEF500809EF6E036A2D51430FE96E5A
:102DE000000E0320EA6EEF50080B0CE0D8902D3552
:102DF000036A5B0FE96E000E0320EA6EEC6AED5287
:102E0000EF6A10D0D8902D35036A5B0FE96E000E83
:102E10000320EA6E000E465D006E080E475900C0A2
:102E2000EFFFEC6E030E7F6F0001DEEC0DF0D8902B
:102E300002012D35036A2B0FE96E000E0320EA6EA6
:102E40003FC2ECFFED523EC2EFFF036A2D51470F28
:102E5000E96E000E0320EA6E48C2EFFF00012CEC81
:102E600007F0010E0201846F000150EC06F08B9216
:102E70008C8085EF19F0186AF2BE188EF29E2EC271
:102E8000B7F22DC2B6F2C5EC00F018BEF28E01C04A
:102E90002FF2020E02012D25336F000E2E21346F0A
:102EA000186AF2BE188EF29EB76F33C2B6F20001F6
:102EB000C5EC00F018BEF28E01C030F202012FC244
:102EC00032F2316B30513127000E322331C201F022
:102ED00032C202F00001000C02012D6B2D510308DB
:102EE00016E3D8902D35036A2B0FE96E000E0320F0
:102EF000EA6E080EEC6EED52EF6A036A2D51470F31
:102F0000E96E000E0320EA6EEF6A2D2BE7D7EA6A1E
:102F1000430EE96EA66BA86B040EA76F0001E1ECEF
:102F200001F0050E02017F6F0001DEEC0DF0EA6A90
:102F3000A90EE96E0201A66BA86B400EA76F0001F7
:102F4000E1EC01F0EA6A690EE96E0201A66BA86B7A
:102F5000400EA76F0001E1EC01F0020E02017F6F4D
:102F60000001DEEC0DF0EA6A5B0EE96E0201A66B71
:102F7000A86B080EA76F0001E1EC01F0030E02013F
:102F80007F6F0001DEEC0DF0010E0201846F000185
:102F900050EC06F02CEC07F04AEF1AF00201406BFF
:102FA000416B010E426FDA6AD96A020E456F380E24
:102FB000446F020EEA6E3C0EE96E45C2E2FF44C267
:102FC000E1FF42C243F2D890E550EE02F3504023B5
:102FD000F4504123432FF7D740C2DEFF41C240F2F5
:102FE000416BD8B0412B442BD8B4452B422B4251D6
:102FF0000508DFE100014FEF18F0020136513803F8
:10300000F3CF01F0F4CF00F03903F350002637512D
:103010003803F3500020026E000175EF18F08E0E99
:10302000006E35C201F034C202F0036A015209E1B8
:1030300002C001F0026A080E005E015202E1006A5D
:1030400008D0D89001BE04D0023601360006F9D768
:10305000019E000CF0832DC2FCF0F66BF56BF46B57
:10306000F36B32C200F0016A026A036A03C037F2EE
:1030700002C036F201C035F232C234F202013B6BBB
:103080003A6B090E396F600E386F03C03FF202C011
:103090003EF201C03DF232C23CF200017FD703C0D4
:1030A000FAF002C0F9F001C0F8F000C0F7F0D890D3
:1030B00002012D35036A2B0FE96E000E0320EA6E24
:1030C000ECCF03F0ED52EFCFF1F0000103C0F2F0CE
:1030D0000201356B33C234F235C237F233C236F2F5
:1030E000396B320E386F000188D702C006F101C07B
:1030F00005F1FB6B0101086B076B020130512E5D7E
:10310000006E31512F59036E00C034F2356F00014B
:1031100086DF00C034F201C035F202C036F203C0CF
:1031200037F203C086F202C085F201C084F200C00B
:1031300083F202018A6B896B886B800E876F0001B6
:10314000A0EC0CF003C000F102C0FFF001C0FEF0E3
:1031500000C0FDF0020130512E25016E31512F21AA
:10316000036E01C034F2356F000159DF00C034F244
:1031700001C035F202C036F203C037F203C086F256
:1031800002C085F201C084F200C083F202018A6BA2
:10319000896B886B800E876F0001A0EC0CF003C078
:1031A00004F102C003F101C002F100C001F1EFEF30
:1031B0001CF0186AF2BE188EF29E010E0201B76F63
:1031C0004E0EB66F0001C5EC00F018BEF28E01C0C5
:1031D0001DF202011D51020A000136E0010A3DE024
:1031E000070A4EE00D0AD8B4A5D0030AD8B41AD104
:1031F000060AD8B427D1010AD8B434D1030AD8B406
:1032000041D1010AD8B44FD11E0AD8B45CD1030A07
:10321000D8B4CAD1010AD8B42AD2060AD8B437D24F
:10322000030AD8B472D2010AD8B484D20F0AD8B42F
:10323000ADD2010AD8B4B3D2030AD8B4B9D2040AC1
:10324000D8B40DD3F8EF1CF002012D6B0001ECECAB
:1032500007F094EC0BF002EF1DF002012D6B000162
:10326000ECEC07F094EC0BF0FDEF0EF0070E020112
:103270002D6F0001ECEC07F094EC0BF002EF1DF069
:103280002992186AF2BE188EF29E010E0201B76FE3
:10329000500EB66F0001C5EC00F018BEF28E01C0F2
:1032A00022F20201225102080AE0010E2D6F0001F4
:1032B000ECEC07F094EC0BF002EF1DF00201186A41
:1032C000F2BE188EF29E010EB76F520EB66F00015D
:1032D000C5EC00F018BEF28E01C021F202012151AE
:1032E000030809E2010E2D6F0001ECEC07F094ECED
:1032F0000BF088D302012D6B0001ECEC07F094EC8D
:103300000BF021C22DF26CEF15F0036A020121517E
:10331000430FE96E000E0320EA6EEF50080B02E146
:103320002A6A2982070E2D6F0001ECEC07F094EC5D
:103330000BF068D3186AF2BE188EF29E010E0201DD
:10334000B76F500EB66F0001C5EC00F018BEF28EDC
:1033500001C022F202012251060809E0010E2D6F80
:103360000001ECEC07F094EC0BF04CD30201186A6E
:10337000F2BE188EF29E010EB76F520EB66F0001AC
:10338000C5EC00F018BEF28E01C021F202012151FD
:10339000030809E2010E2D6F0001ECEC07F094EC3C
:1033A0000BF030D30201010E2E6F540E2D6F000171
:1033B00062DD02C026F201C025F2020126510F088B
:1033C0000EE2FF0A03E12551000809E2010E2D6F0C
:1033D0000001ECEC07F094EC0BF014D302012996F9
:1033E0002D6B0001ECEC07F094EC0BF0D89002018F
:1033F0002135036A2B0FE96E000E0320EA6E26C208
:10340000ECFFED5225C2EFFF010E846F000150EC7E
:1034100006F0070E02012D6F0001ECEC07F094ECB2
:103420000BF0F0D202012D6B0001ECEC07F094ECF4
:103430000BF00B0E02012D6F0001ECEC07F094EC89
:103440000BF0E0D202012D6B0001ECEC07F094ECE4
:103450000BF0080E02012D6F0001ECEC07F094EC6C
:103460000BF0D0D202012D6B0001ECEC07F094ECD4
:103470000BF0060E02012D6F0001ECEC07F094EC4E
:103480000BF0C0D202012D6B0001ECEC07F094ECC4
:103490000BF022D5070E02012D6F0001ECEC07F0B6
:1034A00094EC0BF0AFD202012D6B0001ECEC07F0B5
:1034B00094EC0BF0100E02012D6F0001ECEC07F004
:1034C00094EC0BF09FD2186AF2BE188EF29E010E99
:1034D0000201B76F500EB66F0001C5EC00F018BEC8
:1034E000F28E01C022F202012251020809E0010E0F
:1034F0002D6F0001ECEC07F094EC0BF083D202018D
:10350000186AF2BE188EF29E010EB76F520EB66F99
:103510000001C5EC00F018BEF28E01C023F20201DA
:10352000235132081AE18C860A0E966F010E976FAE
:1035300000014FEC0DF002011E6B1E5103080CE35D
:10354000036A1E51430FE96E000E0320EA6EEF502E
:103550004009EF6E1E2BF1D718D08C960A0E966F8D
:10356000976B00014FEC0DF002011E6B1E5103081A
:103570000CE3036A1E51430FE96E000E0320EA6E4E
:10358000EF50BF0BEF6E1E2BF1D72D6B0001ECEC53
:1035900007F094EC0BF0070E02012D6F0001ECEC2C
:1035A00007F094EC0BF02ED2186AF2BE188EF29E41
:1035B000010E0201B76F500EB66F0001C5EC00F0AE
:1035C00018BEF28E01C022F202012251080809E061
:1035D000010E2D6F0001ECEC07F094EC0BF012D211
:1035E00002011E6B1E51030831E3D8901E35050FF2
:1035F000206F036A20514D0F2D6F010E03202E6F97
:10360000186AF2BE188EF29EB76F2DC2B6F2000194
:10361000C5EC00F018BEF28E01C024F20201245164
:10362000030809E2010E2D6F0001ECEC07F094ECA9
:103630000BF002010BD0036A1E51470FE96E000E1A
:103640000320EA6E24C2EFFF1E2BCCD72D6B0001A6
:10365000ECEC07F094EC0BF02CEC07F0060E0201FA
:103660002D6F0001ECEC07F094EC0BF0CBD10201D4
:103670002D6B0001ECEC07F094EC0BF0140E020142
:103680002D6F0001ECEC07F094EC0BF0BBD1186A45
:10369000F2BE188EF29E010E0201B76F500EB66F89
:1036A0000001C5EC00F018BEF28E01C022F202014A
:1036B0002251040809E0010E2D6F0001ECEC07F027
:1036C00094EC0BF09FD102012D6B0001ECEC07F0A4
:1036D00094EC0BF0010E02012E6F520E2D6F0001C3
:1036E0003BEC17F002C01CF001C01BF0040E0201FD
:1036F0007F6F0001DEEC0DF0100E02012D6F000156
:10370000ECEC07F094EC0BF07DD102012D6B000185
:10371000ECEC07F094EC0BF0F29CF29EF2BEFDD7BD
:10372000D190320E0201986F000114EC07F082EF85
:103730003EF068D129A602D0299601D02986298891
:10374000666A140E656E0F0E646EEC0E636E66C0D4
:1037500068F065C067F002011E6B1E5103080FE39D
:10376000D8901E35036A2B0FE96E000E0320EA6E17
:1037700066C0ECFFED5265C0EFFF1E2BEED72D6B40
:103780000001ECEC07F094EC0BF03CD12980020135
:103790002D6B0001ECEC07F094EC0BF033D1299089
:1037A00002012D6B0001ECEC07F094EC0BF02AD138
:1037B00002011E6B1E5103080AE3036A1E51430FE8
:1037C000E96E000E0320EA6EEF6A1E2BF3D71E6B24
:1037D0001E51030837E31F6B1F51030831E31F51CC
:1037E000100DF3502E6B2D6F1E51040DF350036A14
:1037F0002D25016E2E5103220150690FE96E000E36
:103800000320EA6E7F0EEF6EEC6AEC6AEC6A1F51E1
:10381000100DF3502E6B2D6F1E51040DF350036AE3
:103820002D25016E2E5103220150A90FE96E000EC5
:103830000320EA6EEF6AEC6AEC6AEC6A1F2BCCD7C5
:103840001E2BC6D7020E7F6F0001DEEC0DF00201C9
:103850002D6B0001ECEC07F094EC0BF0D3D0186A60
:10386000F2BE188EF29E010E0201B76F500EB66FB7
:103870000001C5EC00F018BEF28E01C022F2020178
:1038800022510E0809E0010E2D6F0001ECEC07F04B
:1038900094EC0BF0B7D00201186AF2BE188EF29EBB
:1038A000010EB76F520EB66F0001C5EC00F018BEE6
:1038B000F28E01C021F202012151030809E2010E3A
:1038C0002D6F0001ECEC07F094EC0BF09BD00201A3
:1038D000010E2E6F540E2D6F00013BEC17F002C04D
:1038E00028F201C027F2020128510F080EE2FF0A58
:1038F00003E12751000809E2010E2D6F0001ECECF5
:1039000007F094EC0BF07ED00201010E2E6F580EE2
:103910002D6F00013BEC17F002C02AF201C029F222
:10392000020128512A5D0DE303E12951275D09E2D7
:10393000010E2D6F0001ECEC07F094EC0BF062D05F
:103940000201186AF2BE188EF29E010EB76F5C0E6D
:10395000B66F0001C5EC00F018BEF28E01C02CF26B
:1039600002012C51640809E2010E2D6F0001ECECFC
:1039700007F094EC0BF046D00201186AF2BE188EE4
:10398000F29E010EB76F5E0EB66F0001C5EC00F03F
:1039900018BEF28E01C02BF202012B5309E1010E79
:1039A0002D6F0001ECEC07F094EC0BF02BD0020132
:1039B00029962D6B0001ECEC07F094EC0BF021C282
:1039C0002DF228C22FF227C22EF22AC231F229C2CA
:1039D00030F22CC232F22BC233F22AEF18F0070E6B
:1039E00002012D6F0001ECEC07F094EC0BF00AD013
:1039F000010E02012D6F0001ECEC07F0F08D94EC4C
:103A00000BF000D0B9EC00F024EF21F002011D6BA7
:103A10001D51030824E3036A1D51430FE96E000E94
:103A20000320EA6EEF500F0B15E029B213D08B8202
:103A30008C900001F0A504D00101095306E10001BA
:103A4000010E02011D2501010B6F0001F08502012D
:103A500006D003D00001F09502011D2BD9D700013B
:103A6000F0A51FD029B21DD001010A51130803E2AD
:103A70000A6B0BC109F10A2B09530AE00001F0A7F8
:103A800002D0F09701D0F087F0B703D00101090709
:103A90000001F0A703D08B848B9602D08B948B9679
:103AA0000AD08B948B86F0AD04D08B828C90F09DE5
:103AB00002D08B928C805DEF21F002014051D8B48E
:103AC00071D0006E4451D8B46DD0002604E3810E4D
:103AD000002668E204D07F0E005E64E363E041C22A
:103AE00048F24551481B418F458F43514703F4CF5E
:103AF0004AF242514603F4CF03F0F3CF49F24703B1
:103B0000F3504A27F4504923000E03224351460341
:103B1000F3504A27F4504923000E026A032202227E
:103B200041514703F3504927F4500322000E02226B
:103B300041514603F3500326F4500222000E016A5D
:103B4000012243514503F3504927F4500322000E4C
:103B50000222012242514503F3500326F45002226F
:103B6000000E012241514503F3500226F450012278
:103B7000002A01BE05D04937033602360136000659
:103B8000000E49AF0AD0032A02220122015005E1AA
:103B9000025003E1035001E1002A48BF018E48AF03
:103BA000019E04D0006A016A026A036A0001000CE7
:103BB00002014051B608406F036A41C244F2418F8E
:103BC000D890413342334333033202320132003260
:103BD000402FF6D744AF0BD0001E011E021E031E5D
:103BE000002AD8B4012AD8B4022AD8B4032A000182
:103BF00062EF1EF00201216B21510308D8A01AD1F7
:103C0000036A2151470FE96E000E0320EA6EEFCFE1
:103C100023F2D8902135036A2B0FE96E000E0320A2
:103C2000EA6EECCF03F0ED52EFCF38F203C039F279
:103C3000000E385F080E395B39C280F238C27FF25D
:103C4000000178EC0CF000C03AF201C03BF202C077
:103C50003CF203C03DF202012351100DF3503F6BC3
:103C60003E6F2151040DF350036A3E25016E3F5112
:103C700003220150690FE96E000E0320EA6EEFCFB8
:103C800000F0ECCF01F0ECCF02F0ECCF03F03DC23E
:103C900043F23CC242F23BC241F23AC240F203C09C
:103CA00047F202C046F201C045F200C044F20001F2
:103CB00004DF03C043F202C042F201C041F200C07F
:103CC00040F276D703C043F202C042F201C041F293
:103CD00000C040F202012351100DF350456B446FB8
:103CE0002151040DF350036A4425016E455103220E
:103CF0000150A90FE96E000E0320EA6EEFCF00F02D
:103D0000ECCF01F0ECCF02F0ECCF03F000504025F7
:103D1000246F01504121256F02504221266F03502C
:103D20004321276F2151040DF350036A330FE96ECD
:103D3000000E0320EA6EEFCF3AF2ECCF3BF2ECCF6D
:103D40003CF2ECCF3DF23A3D07D03B3D05D03C3D47
:103D500003D03D517F0834E02151040DF350036A34
:103D6000280F016E020E032201C03AF203C03BF29B
:103D70002151040DF350036A330FE96E000E032046
:103D8000EA6EEFCF3CF2ECCF3DF2ECCF3EF2ECCF5F
:103D90003FF224513C5D006E25513D59016E265184
:103DA0003E59026E27513F593BC2EAFF3AC2E9FF32
:103DB00000C0EFFF01C0ECFF02C0ECFFEC6E0FD0C3
:103DC0002151040DF350036A280FE96E020E0320FF
:103DD000EA6EFF0EEF6EEC6EEC6E7F0EEC6E215114
:103DE000040DF350036A330F016E000E032201C06D
:103DF0003AF203C03BF22151040DF350036A280F3D
:103E0000E96E020E0320EA6EEFCF00F0ECCF01F076
:103E1000ECCF02F0ECCF03F03BC2EAFF3AC2E9FF7D
:103E200000C0EFFF01C0ECFF02C0ECFF03C0ECFFDD
:103E3000212BE2D6000160EF21F0050E02012D6F6B
:103E40000001ECEC07F094EC0BF063EF21F0800E36
:103E5000D8A202D00201271B02012C6B2D6B23C2BA
:103E60002BF227512B1B2251D8B4DFD02A6F006EC2
:103E70002651D8B4E3D02A5FD8B483D03EE327C21A
:103E800030F2308F28C22FF229C22EF22D6BD8903B
:103E900030332F332E332D332A2FF8D72BAF03D0C7
:103EA0002C81E0D02C912A912C89020EEA6E250EED
:103EB000E96EEBD02C992BBF0AD02AA113D0303356
:103EC0002F332E332D33002AD8B4C7D00BD030BFB8
:103ED0000CD0D8902D372E372F3730370006D8B476
:103EE000BCD0F5D72C8D6DD02C9D23C22BF223AFE7
:103EF00002D0308FABD0309FA9D026C22AF226C282
:103F000000F022512A5F23C230F2308F24C22FF2F8
:103F100025C22EF22D6BD89030332F332E332D3314
:103F20002A2FF8D72BAF03D02C839CD02C932A9127
:103F30002C8B020EEA6E290EE96EA7D02C9B2BBFAC
:103F40000AD02AA113D030332F332E332D33002A39
:103F5000D8B483D00BD030BF0CD0D8902D372E37AB
:103F60002F3730370006D8B478D0F5D72C8F29D02A
:103F70002C9F27C22BF227AF02D0308F67D0309F03
:103F800065D027C230F2308F28C22FF229C22EF21C
:103F90002BAF04D0309F2C8565D02C952D6B2A91AA
:103FA000020EEA6E250EE96E70D02BBF1CD023C224
:103FB0002BF22AA106D030332F332E332D33002A93
:103FC0004CE02DAF0BD02E2B09E12F2B07E1302B2E
:103FD00005E130332F332E33002A3FE02CBD84D748
:103FE0002CBFC6D71CD0800E301B30AF04D03AD0C7
:103FF00027C22BF20AD023C22BF2305306E12F53F3
:1040000004E12E5302E1006A21D030BF08D0D890DD
:104010002D372E372F373037002EF7D71ED02BAF46
:1040200002D0308F13D0309F11D026C200F027C2AB
:1040300030F228C22FF229C22EF208D022C200F09C
:1040400023C230F224C22FF225C22EF230C201F078
:104050002FC202F02EC203F034D0006A016A026A55
:10406000036A2FD02D6B2E1F2F1F301F2D1F2D2BBE
:1040700005E12E2B03E12F2B01E1302B2CB112D7C0
:104080002CB354D72CB589D7B3D7EF502E2705E3DF
:104090002F2B03E1302BD8B42A81ED52EF502F277C
:1040A00003E3302BD8B42A81ED52EF50EFBE01D09C
:1040B000800A3027D8B02A812CB9FCD62CBB3ED739
:1040C00074D70001EDEF21F08E0E006E02011F513A
:1040D000005E20C202F021C201F0028E005209E00F
:1040E000D890025202E1015204E002320132002E65
:1040F000F7D720AF05D0011E021E012AD8B4022A2C
:10410000000106EF22F0D890FC35036A2B0FE96E10
:10411000000E0320EA6EF2C0ECFFED52F1C0EFFF9B
:10412000010E0201846F000150EC06F08B928C802E
:10413000F09326EF22F0F86AD09E0D8EFE0E006EF0
:10414000060E016E020EE96E000EEA6EEE6A002E99
:10415000FDD7012EFBD7EA6AE96A400EAF6EA60EC4
:10416000AC6E900EAB6EC180C182C184C196196ADB
:104170001A6A020E1D6E040E1E6E060E1F6E080ECB
:10418000206E100E216E120E226E140E236E160E6D
:10419000246E180E256E1A0E266E1C0E276E1E0E2D
:1041A000286EF09D02010F6B106B0001B5EF01F05E
:1041B000F0EF01F0FCEF01F012EF02F08B928C8037
:1041C0008B948B8629902992EA6A430EE96E02014C
:1041D000A66BA86B040EA76F0001E1EC01F0020EC4
:1041E00002011D6F0001B7EC02F0030E02011D6F0A
:1041F0000001B7EC02F0040E02011D6F0001B7ECE4
:1042000002F0050E02011D6F0001B7EC02F04350F1
:10421000400B02E18C9601D08C86010E0201846F66
:10422000000150EC06F02CEC07F00A0E0201986F2A
:10423000000114EC07F0B9EC00F0EDEC03F0040021
:10424000F0A902D0D9EF18F029AC5AD029A632D063
:1042500029A80CD0672AD8B4682A6450685C05E3A2
:1042600003E16350675C01E329980CD06750D8B430
:10427000680667066850665C05E303E16750655CA5
:1042800001E329880201116B115103080FE3D89053
:104290001135036A2B0FE96E000E0320EA6E68C029
:1042A000ECFFED5267C0EFFF112BEED7846B0001DE
:1042B00050EC06F0299C06EF1DF050EC04F09AD467
:1042C00029A001D0BAD529940201116B115103081C
:1042D0000CE3036A1151430FE96E000E0320EA6EEE
:1042E000EF507F0BEF6E112BF1D70001EDEC03F0D7
:1042F00029A206D02A2A2A503C0802E22A6A2992D8
:10430000F0A3A4D0010EF327D8B0F42BD8B4F52B2A
:10431000D8B4F62BFA51F65DD8A098D00EE1F95139
:10432000F55DD8A093D009E1F851F45DD8A08ED006
:1043300004E1F351F75DD8B089D0036AFB51F2CFA5
:104340001DF2F29E5BEC00F002011DBFF28E016EC9
:10435000806B7F6F7FBF8007000178EC0CF000C19D
:1043600043F2FFC042F2FEC041F2FDC040F203C082
:1043700047F202C046F201C045F200C044F25DECD3
:104380001DF000C01EF201C01FF202C020F203C0E7
:1043900021F203C086F202C085F201C084F200C09F
:1043A00083F202018A6B896B7E0E886F850E876FA0
:1043B0000001A0EC0CF0D89204C125F203C124F254
:1043C00002C123F201C122F203C029F202C028F285
:1043D00001C027F200C026F23AD503C018F202C08D
:1043E00017F201C016F200C015F2D890FC35036A2E
:1043F0002B0FE96E000E0320EA6E18C222F217C2DC
:1044000021F216C220F215C21FF25ED602C0ECFFE6
:10441000ED5201C0EFFF0201846B000150EC06F089
:10442000F66BF56BF46BF36BFB2BFB51310801E280
:10443000FB6B0101072BD8B4082B0651085D07E37D
:1044400003E10551075D03E300015DD601010001B1
:04445000F6D6030099
:0200000400F00A
:0A00020000000000000000000000F4
:1000100000080008000800080000000000000000C0
:100080000000000000000000000000000000000070
:100090000000000000000000000000000000000060
:1000A0000000000000000000000000000000000050
:1000B0000000000000000000000000000000000040
:1000C0000000000000000000000000000000000030
:1000D0000000000000000000000000000000000020
:1000E0000000000000000000000000000000000010
:1000F0000000000000000000000000000000000000
:020000040030CA
:00000001FF
